 iterobjreachobj004

 Timestamp is 9d55bb0f (reproducible build file hash)

 Preferred load address is 0000000180000000

 Start         Length     Name                   Class
 0001:00000000 000039d0H .text$mn                CODE
 0001:000039d0 00000036H .text$mn$00             CODE
 0001:00003a06 00000092H .text$x                 CODE
 0002:00000000 000001c8H .idata$5                DATA
 0002:000001c8 00000038H .00cfg                  DATA
 0002:00000200 00000008H .CRT$XCA                DATA
 0002:00000208 00000008H .CRT$XCZ                DATA
 0002:00000210 00000008H .CRT$XIA                DATA
 0002:00000218 00000008H .CRT$XIC                DATA
 0002:00000220 00000008H .CRT$XIZ                DATA
 0002:00000228 00000008H .CRT$XLA                DATA
 0002:00000230 00000008H .CRT$XLZ                DATA
 0002:00000238 00000008H .CRT$XPA                DATA
 0002:00000240 00000008H .CRT$XPZ                DATA
 0002:00000248 00000008H .CRT$XTA                DATA
 0002:00000250 00000010H .CRT$XTZ                DATA
 0002:00000258 00000000H .gehcont$y              DATA
 0002:00000258 00000000H .gfids$y                DATA
 0002:00000260 00002320H .rdata                  DATA
 0002:00002580 00000000H .rdata$CastGuardVftablesA DATA
 0002:00002580 00000000H .rdata$CastGuardVftablesC DATA
 0002:00002580 00000028H .rdata$T                DATA
 0002:000025a8 000000f4H .rdata$voltmd           DATA
 0002:0000269c 00000324H .rdata$zzzdbg           DATA
 0002:000029c0 00000008H .rtc$IAA                DATA
 0002:000029c8 00000008H .rtc$IZZ                DATA
 0002:000029d0 00000008H .rtc$TAA                DATA
 0002:000029d8 00000008H .rtc$TZZ                DATA
 0002:000029e0 00000004H .tls                    DATA
 0002:000029e4 00000004H .tls$                   DATA
 0002:000029e8 00000008H .tls$ZZZ                DATA
 0002:000029f0 00000340H .xdata                  DATA
 0002:00002d30 0000036cH .edata                  DATA
 0002:0000309c 0000008cH .idata$2                DATA
 0002:00003128 00000018H .idata$3                DATA
 0002:00003140 000001c8H .idata$4                DATA
 0002:00003308 00000486H .idata$6                DATA
 0003:00000000 00000090H .data                   DATA
 0003:00000090 0001b248H .bss                    DATA
 0004:00000000 000003ccH .pdata                  DATA

  Address         Publics by Value              Rva+Base               Lib:Object

 0000:00000000       __AbsoluteZero             0000000000000000     <absolute>
 0000:00000000       ___safe_se_handler_count   0000000000000000     <absolute>
 0000:00000000       ___safe_se_handler_table   0000000000000000     <absolute>
 0000:00000000       __arm64x_extra_rfe_table   0000000000000000     <absolute>
 0000:00000000       __arm64x_extra_rfe_table_size 0000000000000000     <absolute>
 0000:00000000       __arm64x_native_entrypoint 0000000000000000     <absolute>
 0000:00000000       __arm64x_redirection_metadata 0000000000000000     <absolute>
 0000:00000000       __arm64x_redirection_metadata_count 0000000000000000     <absolute>
 0000:00000000       __dynamic_value_reloc_table 0000000000000000     <absolute>
 0000:00000000       __enclave_config           0000000000000000     <absolute>
 0000:00000000       __guard_check_icall_a64n_fptr 0000000000000000     <absolute>
 0000:00000000       __guard_eh_cont_count      0000000000000000     <absolute>
 0000:00000000       __guard_eh_cont_table      0000000000000000     <absolute>
 0000:00000000       __guard_fids_count         0000000000000000     <absolute>
 0000:00000000       __guard_fids_table         0000000000000000     <absolute>
 0000:00000000       __guard_iat_count          0000000000000000     <absolute>
 0000:00000000       __guard_iat_table          0000000000000000     <absolute>
 0000:00000000       __guard_longjmp_count      0000000000000000     <absolute>
 0000:00000000       __guard_longjmp_table      0000000000000000     <absolute>
 0000:00000000       __hybrid_auxiliary_iat     0000000000000000     <absolute>
 0000:00000000       __hybrid_auxiliary_iat_copy 0000000000000000     <absolute>
 0000:00000000       __hybrid_code_map          0000000000000000     <absolute>
 0000:00000000       __hybrid_code_map_count    0000000000000000     <absolute>
 0000:00000000       __x64_code_ranges_to_entry_points 0000000000000000     <absolute>
 0000:00000000       __x64_code_ranges_to_entry_points_count 0000000000000000     <absolute>
 0000:00000100       __guard_flags              0000000000000100     <absolute>
 0000:00000000       __ImageBase                0000000180000000     <linker-defined>
 0001:00000000       ?NewObject@JNIEnv_@@QEAAPEAV_jobject@@PEAV_jclass@@PEAU_jmethodID@@ZZ 0000000180001000 f i libiterobjreachobj004.obj
 0001:00000024       ?TranslateError@@YAPEBDW4jvmtiError@@@Z 0000000180001024 f   libiterobjreachobj004.obj
 0001:000002dc       ?nsk_jni_check_exception@@YAHPEAUJNIEnv_@@QEBDH@Z 00000001800012dc f   libiterobjreachobj004.obj
 0001:00000420       ?nsk_jni_lverify@@YAHHPEAUJNIEnv_@@HQEBDH1ZZ 0000000180001420 f   libiterobjreachobj004.obj
 0001:000004c0       Agent_Initialize           00000001800014c0 f   libiterobjreachobj004.obj
 0001:0000069c       Agent_OnAttach             000000018000169c f   libiterobjreachobj004.obj
 0001:0000069c       Agent_OnLoad               000000018000169c f   libiterobjreachobj004.obj
 0001:000006a4       Java_nsk_jvmti_unit_FollowReferences_FollowRefObjects_addRefToVerify 00000001800016a4 f   libiterobjreachobj004.obj
 0001:00000860       Java_nsk_jvmti_unit_FollowReferences_FollowRefObjects_getTag 0000000180001860 f   libiterobjreachobj004.obj
 0001:0000091c       Java_nsk_jvmti_unit_FollowReferences_FollowRefObjects_resetRefsToVerify 000000018000191c f   libiterobjreachobj004.obj
 0001:00000924       Java_nsk_jvmti_unit_FollowReferences_FollowRefObjects_resetTags 0000000180001924 f   libiterobjreachobj004.obj
 0001:00000968       Java_nsk_jvmti_unit_FollowReferences_FollowRefObjects_setTag 0000000180001968 f   libiterobjreachobj004.obj
 0001:00000bb4       Java_nsk_share_jvmti_ArgumentHandler_getAgentOptionsString 0000000180001bb4 f   libiterobjreachobj004.obj
 0001:00000c60       Java_nsk_share_jvmti_DebugeeClass_checkStatus 0000000180001c60 f   libiterobjreachobj004.obj
 0001:00000ce8       Java_nsk_share_jvmti_DebugeeClass_resetAgentData 0000000180001ce8 f   libiterobjreachobj004.obj
 0001:00000d48       Java_nsk_share_jvmti_RedefineAgent_agentStatus 0000000180001d48 f   libiterobjreachobj004.obj
 0001:00000d54       Java_nsk_share_jvmti_RedefineAgent_isRedefined 0000000180001d54 f   libiterobjreachobj004.obj
 0001:00000d60       Java_nsk_share_jvmti_RedefineAgent_redefineAttempted 0000000180001d60 f   libiterobjreachobj004.obj
 0001:00000d6c       MA_checkStatus             0000000180001d6c f   libiterobjreachobj004.obj
 0001:00000e10       __local_stdio_printf_options 0000000180001e10 f i libiterobjreachobj004.obj
 0001:0000153c       exitOnError                000000018000253c f   libiterobjreachobj004.obj
 0001:000015f0       fprintf                    00000001800025f0 f i libiterobjreachobj004.obj
 0001:00001634       nsk_complain               0000000180002634 f   libiterobjreachobj004.obj
 0001:00001660       nsk_jvmti_classBySignature 0000000180002660 f   libiterobjreachobj004.obj
 0001:00001a14       nsk_jvmti_createJVMTIEnv   0000000180002a14 f   libiterobjreachobj004.obj
 0001:00001b44       nsk_jvmti_lverify          0000000180002b44 f   libiterobjreachobj004.obj
 0001:00001c34       nsk_jvmti_parseOptions     0000000180002c34 f   libiterobjreachobj004.obj
 0001:00001e84       nsk_jvmti_resetAgentData   0000000180002e84 f   libiterobjreachobj004.obj
 0001:00001ef8       nsk_jvmti_resumeSync       0000000180002ef8 f   libiterobjreachobj004.obj
 0001:00001f9c       nsk_jvmti_waitForSync      0000000180002f9c f   libiterobjreachobj004.obj
 0001:000020a0       nsk_lcomplain              00000001800030a0 f   libiterobjreachobj004.obj
 0001:000020c0       nsk_ldisplay               00000001800030c0 f   libiterobjreachobj004.obj
 0001:000020e0       nsk_ltrace                 00000001800030e0 f   libiterobjreachobj004.obj
 0001:00002100       nsk_lvcomplain             0000000180003100 f   libiterobjreachobj004.obj
 0001:000022b8       nsk_lvdisplay              00000001800032b8 f   libiterobjreachobj004.obj
 0001:00002304       nsk_lverify                0000000180003304 f   libiterobjreachobj004.obj
 0001:00002360       nsk_lvtrace                0000000180003360 f   libiterobjreachobj004.obj
 0001:000023c0       nsk_printf                 00000001800033c0 f   libiterobjreachobj004.obj
 0001:000023e8       nsk_vprintf                00000001800033e8 f   libiterobjreachobj004.obj
 0001:0000249c       objectReferenceCallback    000000018000349c f   libiterobjreachobj004.obj
 0001:000025a4       printf                     00000001800035a4 f i libiterobjreachobj004.obj
 0001:00002aa4       __raise_securityfailure    0000000180003aa4 f   MSVCRT:gs_report.obj
 0001:00002ad8       __report_gsfailure         0000000180003ad8 f   MSVCRT:gs_report.obj
 0001:00002d18       __GSHandlerCheck           0000000180003d18 f   MSVCRT:gshandler.obj
 0001:00002d38       __GSHandlerCheckCommon     0000000180003d38 f   MSVCRT:gshandler.obj
 0001:00002db0       __security_check_cookie    0000000180003db0 f   MSVCRT:amdsecgs.obj
 0001:000030f0       _DllMainCRTStartup         00000001800040f0 f   MSVCRT:dll_dllmain.obj
 0001:00003130       __scrt_acquire_startup_lock 0000000180004130 f   MSVCRT:utility.obj
 0001:0000316c       __scrt_dllmain_after_initialize_c 000000018000416c f   MSVCRT:utility.obj
 0001:000031a0       __scrt_dllmain_before_initialize_c 00000001800041a0 f   MSVCRT:utility.obj
 0001:000031b8       __scrt_dllmain_crt_thread_attach 00000001800041b8 f   MSVCRT:utility.obj
 0001:000031e0       __scrt_dllmain_crt_thread_detach 00000001800041e0 f   MSVCRT:utility.obj
 0001:000031f8       __scrt_dllmain_exception_filter 00000001800041f8 f   MSVCRT:utility.obj
 0001:00003258       __scrt_dllmain_uninitialize_c 0000000180004258 f   MSVCRT:utility.obj
 0001:00003288       __scrt_dllmain_uninitialize_critical 0000000180004288 f   MSVCRT:utility.obj
 0001:0000329c       __scrt_initialize_crt      000000018000429c f   MSVCRT:utility.obj
 0001:000032e8       __scrt_initialize_onexit_tables 00000001800042e8 f   MSVCRT:utility.obj
 0001:00003374       __scrt_is_nonwritable_in_current_image 0000000180004374 f   MSVCRT:utility.obj
 0001:0000340c       __scrt_release_startup_lock 000000018000440c f   MSVCRT:utility.obj
 0001:00003430       __scrt_uninitialize_crt    0000000180004430 f   MSVCRT:utility.obj
 0001:0000345c       _onexit                    000000018000445c f   MSVCRT:utility.obj
 0001:00003498       atexit                     0000000180004498 f   MSVCRT:utility.obj
 0001:000034b0       __crt_debugger_hook        00000001800044b0 f   MSVCRT:utility_desktop.obj
 0001:000034b8       __scrt_fastfail            00000001800044b8 f   MSVCRT:utility_desktop.obj
 0001:00003604       _guard_check_icall_nop     0000000180004604 f i MSVCRT:guard_support.obj
 0001:00003608       __security_init_cookie     0000000180004608 f   MSVCRT:gs_support.obj
 0001:000036b4       DllMain                    00000001800046b4 f   MSVCRT:dll_dllmain_stub.obj
 0001:000036d8       ?__scrt_initialize_type_info@@YAXXZ 00000001800046d8 f   MSVCRT:tncleanup.obj
 0001:000036e8       ?__scrt_uninitialize_type_info@@YAXXZ 00000001800046e8 f   MSVCRT:tncleanup.obj
 0001:000036f4       __local_stdio_scanf_options 00000001800046f4 f i MSVCRT:default_local_stdio_options.obj
 0001:000036fc       __scrt_initialize_default_local_stdio_options 00000001800046fc f   MSVCRT:default_local_stdio_options.obj
 0001:00003718       __scrt_get_dyn_tls_init_callback 0000000180004718 f   MSVCRT:dyn_tls_init.obj
 0001:00003720       _RTC_Initialize            0000000180004720 f   MSVCRT:initsect.obj
 0001:0000375c       _RTC_Terminate             000000018000475c f   MSVCRT:initsect.obj
 0001:00003798       __isa_available_init       0000000180004798 f   MSVCRT:cpu_disp.obj
 0001:00003944       _get_startup_argv_mode     0000000180004944 f   MSVCRT:argv_mode.obj
 0001:0000394c       __scrt_is_ucrt_dll_in_use  000000018000494c f   MSVCRT:ucrt_detection.obj
 0001:00003960       memcpy                     0000000180004960 f   vcruntime:VCRUNTIME140.dll
 0001:00003966       memset                     0000000180004966 f   vcruntime:VCRUNTIME140.dll
 0001:0000396c       strchr                     000000018000496c f   vcruntime:VCRUNTIME140.dll
 0001:00003972       __C_specific_handler       0000000180004972 f   vcruntime:VCRUNTIME140.dll
 0001:00003978       __std_type_info_destroy_list 0000000180004978 f   vcruntime:VCRUNTIME140.dll
 0001:0000397e       strcmp                     000000018000497e f   ucrt:api-ms-win-crt-string-l1-1-0.dll
 0001:00003984       strlen                     0000000180004984 f   ucrt:api-ms-win-crt-string-l1-1-0.dll
 0001:0000398a       _initterm                  000000018000498a f   ucrt:api-ms-win-crt-runtime-l1-1-0.dll
 0001:00003990       _initterm_e                0000000180004990 f   ucrt:api-ms-win-crt-runtime-l1-1-0.dll
 0001:00003996       _seh_filter_dll            0000000180004996 f   ucrt:api-ms-win-crt-runtime-l1-1-0.dll
 0001:0000399c       _configure_narrow_argv     000000018000499c f   ucrt:api-ms-win-crt-runtime-l1-1-0.dll
 0001:000039a2       _initialize_narrow_environment 00000001800049a2 f   ucrt:api-ms-win-crt-runtime-l1-1-0.dll
 0001:000039a8       _initialize_onexit_table   00000001800049a8 f   ucrt:api-ms-win-crt-runtime-l1-1-0.dll
 0001:000039ae       _register_onexit_function  00000001800049ae f   ucrt:api-ms-win-crt-runtime-l1-1-0.dll
 0001:000039b4       _execute_onexit_table      00000001800049b4 f   ucrt:api-ms-win-crt-runtime-l1-1-0.dll
 0001:000039ba       _crt_atexit                00000001800049ba f   ucrt:api-ms-win-crt-runtime-l1-1-0.dll
 0001:000039c0       _cexit                     00000001800049c0 f   ucrt:api-ms-win-crt-runtime-l1-1-0.dll
 0001:000039c8       __acrt_initialize          00000001800049c8 f   MSVCRT:ucrt_stubs.obj
 0001:000039c8       __acrt_thread_attach       00000001800049c8 f   MSVCRT:ucrt_stubs.obj
 0001:000039c8       __acrt_thread_detach       00000001800049c8 f   MSVCRT:ucrt_stubs.obj
 0001:000039c8       __acrt_uninitialize        00000001800049c8 f   MSVCRT:ucrt_stubs.obj
 0001:000039c8       __acrt_uninitialize_critical 00000001800049c8 f   MSVCRT:ucrt_stubs.obj
 0001:000039c8       __scrt_stub_for_acrt_initialize 00000001800049c8 f   MSVCRT:ucrt_stubs.obj
 0001:000039c8       __scrt_stub_for_acrt_thread_attach 00000001800049c8 f   MSVCRT:ucrt_stubs.obj
 0001:000039c8       __scrt_stub_for_acrt_thread_detach 00000001800049c8 f   MSVCRT:ucrt_stubs.obj
 0001:000039c8       __scrt_stub_for_acrt_uninitialize 00000001800049c8 f   MSVCRT:ucrt_stubs.obj
 0001:000039c8       __scrt_stub_for_acrt_uninitialize_critical 00000001800049c8 f   MSVCRT:ucrt_stubs.obj
 0001:000039c8       __vcrt_initialize          00000001800049c8 f   MSVCRT:ucrt_stubs.obj
 0001:000039c8       __vcrt_thread_attach       00000001800049c8 f   MSVCRT:ucrt_stubs.obj
 0001:000039c8       __vcrt_thread_detach       00000001800049c8 f   MSVCRT:ucrt_stubs.obj
 0001:000039c8       __vcrt_uninitialize        00000001800049c8 f   MSVCRT:ucrt_stubs.obj
 0001:000039c8       __vcrt_uninitialize_critical 00000001800049c8 f   MSVCRT:ucrt_stubs.obj
 0001:000039cc       __scrt_stub_for_is_c_termination_complete 00000001800049cc f   MSVCRT:ucrt_stubs.obj
 0001:000039cc       _is_c_termination_complete 00000001800049cc f   MSVCRT:ucrt_stubs.obj
 0001:000039e0       _guard_dispatch_icall_nop  00000001800049e0 f   MSVCRT:guard_dispatch.obj
 0001:00003a00       _guard_xfg_dispatch_icall_nop 0000000180004a00 f   MSVCRT:guard_xfg_dispatch.obj
 0002:00000000       __imp_RtlCaptureContext    0000000180005000     kernel32:KERNEL32.dll
 0002:00000008       __imp_RtlLookupFunctionEntry 0000000180005008     kernel32:KERNEL32.dll
 0002:00000010       __imp_RtlVirtualUnwind     0000000180005010     kernel32:KERNEL32.dll
 0002:00000018       __imp_UnhandledExceptionFilter 0000000180005018     kernel32:KERNEL32.dll
 0002:00000020       __imp_SetUnhandledExceptionFilter 0000000180005020     kernel32:KERNEL32.dll
 0002:00000028       __imp_GetCurrentProcess    0000000180005028     kernel32:KERNEL32.dll
 0002:00000030       __imp_TerminateProcess     0000000180005030     kernel32:KERNEL32.dll
 0002:00000038       __imp_IsProcessorFeaturePresent 0000000180005038     kernel32:KERNEL32.dll
 0002:00000040       __imp_CloseHandle          0000000180005040     kernel32:KERNEL32.dll
 0002:00000048       __imp_InitializeCriticalSectionAndSpinCount 0000000180005048     kernel32:KERNEL32.dll
 0002:00000050       __imp_DeleteCriticalSection 0000000180005050     kernel32:KERNEL32.dll
 0002:00000058       __imp_CreateEventW         0000000180005058     kernel32:KERNEL32.dll
 0002:00000060       __imp_GetModuleHandleW     0000000180005060     kernel32:KERNEL32.dll
 0002:00000068       __imp_GetProcAddress       0000000180005068     kernel32:KERNEL32.dll
 0002:00000070       __imp_IsDebuggerPresent    0000000180005070     kernel32:KERNEL32.dll
 0002:00000078       __imp_QueryPerformanceCounter 0000000180005078     kernel32:KERNEL32.dll
 0002:00000080       __imp_GetCurrentProcessId  0000000180005080     kernel32:KERNEL32.dll
 0002:00000088       __imp_GetCurrentThreadId   0000000180005088     kernel32:KERNEL32.dll
 0002:00000090       __imp_GetSystemTimeAsFileTime 0000000180005090     kernel32:KERNEL32.dll
 0002:00000098       __imp_DisableThreadLibraryCalls 0000000180005098     kernel32:KERNEL32.dll
 0002:000000a0       __imp_InitializeSListHead  00000001800050a0     kernel32:KERNEL32.dll
 0002:000000a8       \177KERNEL32_NULL_THUNK_DATA 00000001800050a8     kernel32:KERNEL32.dll
 0002:000000b0       __imp_memcpy               00000001800050b0     vcruntime:VCRUNTIME140.dll
 0002:000000b8       __imp_memset               00000001800050b8     vcruntime:VCRUNTIME140.dll
 0002:000000c0       __imp_strchr               00000001800050c0     vcruntime:VCRUNTIME140.dll
 0002:000000c8       __imp___C_specific_handler 00000001800050c8     vcruntime:VCRUNTIME140.dll
 0002:000000d0       __imp___std_type_info_destroy_list 00000001800050d0     vcruntime:VCRUNTIME140.dll
 0002:000000d8       \177VCRUNTIME140_NULL_THUNK_DATA 00000001800050d8     vcruntime:VCRUNTIME140.dll
 0002:000000e0       __imp_strtol               00000001800050e0     ucrt:api-ms-win-crt-convert-l1-1-0.dll
 0002:000000e8       \177api-ms-win-crt-convert-l1-1-0_NULL_THUNK_DATA 00000001800050e8     ucrt:api-ms-win-crt-convert-l1-1-0.dll
 0002:000000f0       __imp_malloc               00000001800050f0     ucrt:api-ms-win-crt-heap-l1-1-0.dll
 0002:000000f8       __imp_free                 00000001800050f8     ucrt:api-ms-win-crt-heap-l1-1-0.dll
 0002:00000100       \177api-ms-win-crt-heap-l1-1-0_NULL_THUNK_DATA 0000000180005100     ucrt:api-ms-win-crt-heap-l1-1-0.dll
 0002:00000108       __imp__errno               0000000180005108     ucrt:api-ms-win-crt-runtime-l1-1-0.dll
 0002:00000110       __imp_exit                 0000000180005110     ucrt:api-ms-win-crt-runtime-l1-1-0.dll
 0002:00000118       __imp__cexit               0000000180005118     ucrt:api-ms-win-crt-runtime-l1-1-0.dll
 0002:00000120       __imp__crt_atexit          0000000180005120     ucrt:api-ms-win-crt-runtime-l1-1-0.dll
 0002:00000128       __imp__execute_onexit_table 0000000180005128     ucrt:api-ms-win-crt-runtime-l1-1-0.dll
 0002:00000130       __imp__register_onexit_function 0000000180005130     ucrt:api-ms-win-crt-runtime-l1-1-0.dll
 0002:00000138       __imp__initialize_onexit_table 0000000180005138     ucrt:api-ms-win-crt-runtime-l1-1-0.dll
 0002:00000140       __imp__initialize_narrow_environment 0000000180005140     ucrt:api-ms-win-crt-runtime-l1-1-0.dll
 0002:00000148       __imp__configure_narrow_argv 0000000180005148     ucrt:api-ms-win-crt-runtime-l1-1-0.dll
 0002:00000150       __imp__seh_filter_dll      0000000180005150     ucrt:api-ms-win-crt-runtime-l1-1-0.dll
 0002:00000158       __imp__initterm_e          0000000180005158     ucrt:api-ms-win-crt-runtime-l1-1-0.dll
 0002:00000160       __imp__initterm            0000000180005160     ucrt:api-ms-win-crt-runtime-l1-1-0.dll
 0002:00000168       \177api-ms-win-crt-runtime-l1-1-0_NULL_THUNK_DATA 0000000180005168     ucrt:api-ms-win-crt-runtime-l1-1-0.dll
 0002:00000170       __imp___acrt_iob_func      0000000180005170     ucrt:api-ms-win-crt-stdio-l1-1-0.dll
 0002:00000178       __imp_fflush               0000000180005178     ucrt:api-ms-win-crt-stdio-l1-1-0.dll
 0002:00000180       __imp___stdio_common_vsprintf 0000000180005180     ucrt:api-ms-win-crt-stdio-l1-1-0.dll
 0002:00000188       __imp___stdio_common_vfprintf 0000000180005188     ucrt:api-ms-win-crt-stdio-l1-1-0.dll
 0002:00000190       \177api-ms-win-crt-stdio-l1-1-0_NULL_THUNK_DATA 0000000180005190     ucrt:api-ms-win-crt-stdio-l1-1-0.dll
 0002:00000198       __imp_strcmp               0000000180005198     ucrt:api-ms-win-crt-string-l1-1-0.dll
 0002:000001a0       __imp__strdup              00000001800051a0     ucrt:api-ms-win-crt-string-l1-1-0.dll
 0002:000001a0       __imp_strdup               00000001800051a0     ucrt:api-ms-win-crt-string-l1-1-0.dll
 0002:000001a8       __imp_strlen               00000001800051a8     ucrt:api-ms-win-crt-string-l1-1-0.dll
 0002:000001b0       __imp_strpbrk              00000001800051b0     ucrt:api-ms-win-crt-string-l1-1-0.dll
 0002:000001b8       __imp_strncpy              00000001800051b8     ucrt:api-ms-win-crt-string-l1-1-0.dll
 0002:000001c0       \177api-ms-win-crt-string-l1-1-0_NULL_THUNK_DATA 00000001800051c0     ucrt:api-ms-win-crt-string-l1-1-0.dll
 0002:000001c8       __guard_check_icall_fptr   00000001800051c8     MSVCRT:guard_support.obj
 0002:000001d0       __guard_xfg_check_icall_fptr 00000001800051d0     MSVCRT:guard_support.obj
 0002:000001d8       __guard_dispatch_icall_fptr 00000001800051d8     MSVCRT:guard_support.obj
 0002:000001e0       __guard_xfg_dispatch_icall_fptr 00000001800051e0     MSVCRT:guard_support.obj
 0002:000001e8       __guard_xfg_table_dispatch_icall_fptr 00000001800051e8     MSVCRT:guard_support.obj
 0002:000001f0       __castguard_check_failure_os_handled_fptr 00000001800051f0     MSVCRT:guard_support.obj
 0002:000001f8       __guard_memcpy_fptr        00000001800051f8     vcruntime:softmemtag.obj
 0002:00000200       __xc_a                     0000000180005200     MSVCRT:initializers.obj
 0002:00000208       __xc_z                     0000000180005208     MSVCRT:initializers.obj
 0002:00000210       __xi_a                     0000000180005210     MSVCRT:initializers.obj
 0002:00000220       __xi_z                     0000000180005220     MSVCRT:initializers.obj
 0002:00000228       __xl_a                     0000000180005228     MSVCRT:tlssup.obj
 0002:00000230       __xl_z                     0000000180005230     MSVCRT:tlssup.obj
 0002:00000238       __xp_a                     0000000180005238     MSVCRT:initializers.obj
 0002:00000240       __xp_z                     0000000180005240     MSVCRT:initializers.obj
 0002:00000248       __xt_a                     0000000180005248     MSVCRT:initializers.obj
 0002:00000250       __xt_z                     0000000180005250     MSVCRT:initializers.obj
 0002:00000260       g_refKindStr               0000000180005260     libiterobjreachobj004.obj
 0002:00000410       ??_C@_09BPLDFGCI@unknown_0@ 0000000180005410     libiterobjreachobj004.obj
 0002:00000420       ??_C@_0BL@FPNMECJD@JVMTI_HEAP_REFERENCE_CLASS@ 0000000180005420     libiterobjreachobj004.obj
 0002:00000440       ??_C@_0BL@FKGKKLNM@JVMTI_HEAP_REFERENCE_FIELD@ 0000000180005440     libiterobjreachobj004.obj
 0002:00000460       ??_C@_0CD@CAEHCFJF@JVMTI_HEAP_REFERENCE_ARRAY_ELEM@ 0000000180005460     libiterobjreachobj004.obj
 0002:00000488       ??_C@_0CC@DNEBMCNK@JVMTI_HEAP_REFERENCE_CLASS_LOAD@ 0000000180005488     libiterobjreachobj004.obj
 0002:000004b0       ??_C@_0BN@CJMIPEBB@JVMTI_HEAP_REFERENCE_SIGNERS@ 00000001800054b0     libiterobjreachobj004.obj
 0002:000004d0       ??_C@_0CH@HBOIDPEB@JVMTI_HEAP_REFERENCE_PROTECTION@ 00000001800054d0     libiterobjreachobj004.obj
 0002:000004f8       ??_C@_0BP@MDKGDGKL@JVMTI_HEAP_REFERENCE_INTERFACE@ 00000001800054f8     libiterobjreachobj004.obj
 0002:00000518       ??_C@_0CC@JJMIHNJH@JVMTI_HEAP_REFERENCE_STATIC_FIE@ 0000000180005518     libiterobjreachobj004.obj
 0002:00000540       ??_C@_0CD@IDHEEGID@JVMTI_HEAP_REFERENCE_CONSTANT_P@ 0000000180005540     libiterobjreachobj004.obj
 0002:00000568       ??_C@_0CA@EFFCHNG@JVMTI_HEAP_REFERENCE_SUPERCLASS@ 0000000180005568     libiterobjreachobj004.obj
 0002:00000588       ??_C@_0L@PCDFHGCJ@unknown_11@ 0000000180005588     libiterobjreachobj004.obj
 0002:00000598       ??_C@_0L@NJBICFOK@unknown_12@ 0000000180005598     libiterobjreachobj004.obj
 0002:000005a8       ??_C@_0L@MAADBEKL@unknown_13@ 00000001800055a8     libiterobjreachobj004.obj
 0002:000005b8       ??_C@_0L@IPECICGM@unknown_14@ 00000001800055b8     libiterobjreachobj004.obj
 0002:000005c8       ??_C@_0L@JGFJLDCN@unknown_15@ 00000001800055c8     libiterobjreachobj004.obj
 0002:000005d8       ??_C@_0L@LNHEOAOO@unknown_16@ 00000001800055d8     libiterobjreachobj004.obj
 0002:000005e8       ??_C@_0L@KEGPNBKP@unknown_17@ 00000001800055e8     libiterobjreachobj004.obj
 0002:000005f8       ??_C@_0L@CDPHMNGA@unknown_18@ 00000001800055f8     libiterobjreachobj004.obj
 0002:00000608       ??_C@_0L@DKOMPMCB@unknown_19@ 0000000180005608     libiterobjreachobj004.obj
 0002:00000618       ??_C@_0L@OJGIPJDB@unknown_20@ 0000000180005618     libiterobjreachobj004.obj
 0002:00000628       ??_C@_0CA@KAOFNDEM@JVMTI_HEAP_REFERENCE_JNI_GLOBAL@ 0000000180005628     libiterobjreachobj004.obj
 0002:00000648       ??_C@_0CC@HPFAJBK@JVMTI_HEAP_REFERENCE_SYSTEM_CLA@ 0000000180005648     libiterobjreachobj004.obj
 0002:00000670       ??_C@_0BN@FDEGFOHC@JVMTI_HEAP_REFERENCE_MONITOR@ 0000000180005670     libiterobjreachobj004.obj
 0002:00000690       ??_C@_0CB@HKIBCMAJ@JVMTI_HEAP_REFERENCE_STACK_LOCA@ 0000000180005690     libiterobjreachobj004.obj
 0002:000006b8       ??_C@_0BP@EAACMMOE@JVMTI_HEAP_REFERENCE_JNI_LOCAL@ 00000001800056b8     libiterobjreachobj004.obj
 0002:000006d8       ??_C@_0BM@IJDEOGOE@JVMTI_HEAP_REFERENCE_THREAD@ 00000001800056d8     libiterobjreachobj004.obj
 0002:000006f8       ??_C@_0BL@EDGPPKC@JVMTI_HEAP_REFERENCE_OTHER@ 00000001800056f8     libiterobjreachobj004.obj
 0002:00000714       ??_C@_04BCJPDBDA@Code@     0000000180005714     libiterobjreachobj004.obj
 0002:00000720       ??_C@_0BA@OCLMCFKC@LineNumberTable@ 0000000180005720     libiterobjreachobj004.obj
 0002:00000730       ??_C@_0BD@CPAEPILC@LocalVariableTable@ 0000000180005730     libiterobjreachobj004.obj
 0002:00000748       ??_C@_0BH@NMBDNHBD@LocalVariableTypeTable@ 0000000180005748     libiterobjreachobj004.obj
 0002:00000760       ??_C@_0O@HIHEEDNJ@StackMapTable@ 0000000180005760     libiterobjreachobj004.obj
 0002:00000770       ??_C@_0BD@BKLAPADN@local_storage_data@ 0000000180005770     libiterobjreachobj004.obj
 0002:00000790       ??_C@_0EF@FGKEPMPL@Lnsk?1jvmti?1IterateOverObjectsRe@ 0000000180005790     libiterobjreachobj004.obj
 0002:000007d8       ??_C@_06IEOJBDIK@object@   00000001800057d8     libiterobjreachobj004.obj
 0002:000007e0       ??_C@_0L@HCDIAMJG@?9?5?$CFs?0?5?$CFd?3?5@ 00000001800057e0     libiterobjreachobj004.obj
 0002:000007f0       ??_C@_0JI@HLPECLFI@?$CD?5?4?4?4?6?$CD?5ERROR?3?5too?5many?5complai@ 00000001800057f0     libiterobjreachobj004.obj
 0002:00000890       ??_C@_0ED@JNEKCCOB@The?5following?5fake?5exception?5st@ 0000000180005890     libiterobjreachobj004.obj
 0002:000008d8       ??_C@_0CN@FCNMDFBH@nsk?4share?4Fake_Exception_for_RU@ 00000001800058d8     libiterobjreachobj004.obj
 0002:00000908       ??_C@_08PGFFNAEI@?$CI?$CFs?3?$CFd?$CJ?5@ 0000000180005908     libiterobjreachobj004.obj
 0002:00000918       ??_C@_0DP@IENMAEGI@s?2test?2hotspot?2jtreg?2vmTestbase@ 0000000180005918     libiterobjreachobj004.obj
 0002:00000958       ??_C@_0BL@NDJLFFJB@?7at?5nsk_lvcomplain?$CI?$CFs?3?$CFd?$CJ?6@ 0000000180005958     libiterobjreachobj004.obj
 0002:00000978       ??_C@_0BC@JOOKAFKF@?$CD?5ERROR?3?5?$CFs?0?5?$CFd?3?5@ 0000000180005978     libiterobjreachobj004.obj
 0002:00000990       ??_C@_09KJEAHMEH@?$CD?5ERROR?3?5@ 0000000180005990     libiterobjreachobj004.obj
 0002:0000099c       ??_C@_02GPIOPFAK@?$DO?$DO@ 000000018000599c     libiterobjreachobj004.obj
 0002:000009a0       ??_C@_02FODMEDOG@?$DM?$DM@ 00000001800059a0     libiterobjreachobj004.obj
 0002:000009a4       ??_C@_02DJGKEECL@?4?4@     00000001800059a4     libiterobjreachobj004.obj
 0002:000009a8       ??_C@_0O@CJPGJOAF@?9?5?$CFs?0?5?$CFd?3?5?$CFs?5@ 00000001800059a8     libiterobjreachobj004.obj
 0002:000009b8       ??_C@_0CB@IAKPDOIC@?$CD?5?5?5verified?5assertion?5is?5FALSE@ 00000001800059b8     libiterobjreachobj004.obj
 0002:000009e0       ??_C@_0CO@LGONDEPD@stdout?3?5fflush?5failed?5?9?5err?$DN?$CFd?5@ 00000001800059e0     libiterobjreachobj004.obj
 0002:00000a10       ??_C@_0CO@KBGKJPBD@stderr?3?5fflush?5failed?5?9?5err?$DN?$CFd?5@ 0000000180005a10     libiterobjreachobj004.obj
 0002:00000a40       ??_C@_0BB@JCNMKLLK@JVMTI_ERROR_NONE@ 0000000180005a40     libiterobjreachobj004.obj
 0002:00000a58       ??_C@_0BL@LDIMKLPH@JVMTI_ERROR_INVALID_THREAD@ 0000000180005a58     libiterobjreachobj004.obj
 0002:00000a78       ??_C@_0CB@PJFPAIKJ@JVMTI_ERROR_INVALID_THREAD_GROU@ 0000000180005a78     libiterobjreachobj004.obj
 0002:00000aa0       ??_C@_0BN@LLMKHMNF@JVMTI_ERROR_INVALID_PRIORITY@ 0000000180005aa0     libiterobjreachobj004.obj
 0002:00000ac0       ??_C@_0CB@MBOFKAGB@JVMTI_ERROR_THREAD_NOT_SUSPENDE@ 0000000180005ac0     libiterobjreachobj004.obj
 0002:00000ae8       ??_C@_0BN@FABOLPBI@JVMTI_ERROR_THREAD_SUSPENDED@ 0000000180005ae8     libiterobjreachobj004.obj
 0002:00000b08       ??_C@_0BN@FDGNOBJM@JVMTI_ERROR_THREAD_NOT_ALIVE@ 0000000180005b08     libiterobjreachobj004.obj
 0002:00000b28       ??_C@_0BL@GOBIFKNJ@JVMTI_ERROR_INVALID_OBJECT@ 0000000180005b28     libiterobjreachobj004.obj
 0002:00000b48       ??_C@_0BK@FCMAJPPC@JVMTI_ERROR_INVALID_CLASS@ 0000000180005b48     libiterobjreachobj004.obj
 0002:00000b68       ??_C@_0BP@IKLLBKEB@JVMTI_ERROR_CLASS_NOT_PREPARED@ 0000000180005b68     libiterobjreachobj004.obj
 0002:00000b88       ??_C@_0BN@KLPPLKG@JVMTI_ERROR_INVALID_METHODID@ 0000000180005b88     libiterobjreachobj004.obj
 0002:00000ba8       ??_C@_0BN@BCEKOKND@JVMTI_ERROR_INVALID_LOCATION@ 0000000180005ba8     libiterobjreachobj004.obj
 0002:00000bc8       ??_C@_0BM@DFDGPME@JVMTI_ERROR_INVALID_FIELDID@ 0000000180005bc8     libiterobjreachobj004.obj
 0002:00000be8       ??_C@_0BL@NELIEPEC@JVMTI_ERROR_NO_MORE_FRAMES@ 0000000180005be8     libiterobjreachobj004.obj
 0002:00000c08       ??_C@_0BJ@BDBECFDM@JVMTI_ERROR_OPAQUE_FRAME@ 0000000180005c08     libiterobjreachobj004.obj
 0002:00000c28       ??_C@_0BK@MIIFNLOB@JVMTI_ERROR_TYPE_MISMATCH@ 0000000180005c28     libiterobjreachobj004.obj
 0002:00000c48       ??_C@_0BJ@HPCAOILC@JVMTI_ERROR_INVALID_SLOT@ 0000000180005c48     libiterobjreachobj004.obj
 0002:00000c68       ??_C@_0BG@CHILOPNI@JVMTI_ERROR_DUPLICATE@ 0000000180005c68     libiterobjreachobj004.obj
 0002:00000c80       ??_C@_0BG@DIEMLHKM@JVMTI_ERROR_NOT_FOUND@ 0000000180005c80     libiterobjreachobj004.obj
 0002:00000c98       ??_C@_0BM@NHMCKHOB@JVMTI_ERROR_INVALID_MONITOR@ 0000000180005c98     libiterobjreachobj004.obj
 0002:00000cb8       ??_C@_0BO@PPEDAJGL@JVMTI_ERROR_NOT_MONITOR_OWNER@ 0000000180005cb8     libiterobjreachobj004.obj
 0002:00000cd8       ??_C@_0BG@FCAIPEID@JVMTI_ERROR_INTERRUPT@ 0000000180005cd8     libiterobjreachobj004.obj
 0002:00000cf0       ??_C@_0CB@EGDBNKOI@JVMTI_ERROR_INVALID_CLASS_FORMA@ 0000000180005cf0     libiterobjreachobj004.obj
 0002:00000d18       ??_C@_0CG@DGKOGIAL@JVMTI_ERROR_CIRCULAR_CLASS_DEFI@ 0000000180005d18     libiterobjreachobj004.obj
 0002:00000d40       ??_C@_0BP@ICEALPKC@JVMTI_ERROR_FAILS_VERIFICATION@ 0000000180005d40     libiterobjreachobj004.obj
 0002:00000d60       ??_C@_0DC@JDACLMIO@JVMTI_ERROR_UNSUPPORTED_REDEFIN@ 0000000180005d60     libiterobjreachobj004.obj
 0002:00000d98       ??_C@_0DE@GKDKNOMJ@JVMTI_ERROR_UNSUPPORTED_REDEFIN@ 0000000180005d98     libiterobjreachobj004.obj
 0002:00000dd0       ??_C@_0BO@LAFKIOG@JVMTI_ERROR_INVALID_TYPESTATE@ 0000000180005dd0     libiterobjreachobj004.obj
 0002:00000df0       ??_C@_0DH@INDGCLLB@JVMTI_ERROR_UNSUPPORTED_REDEFIN@ 0000000180005df0     libiterobjreachobj004.obj
 0002:00000e28       ??_C@_0DE@NHEOMMGI@JVMTI_ERROR_UNSUPPORTED_REDEFIN@ 0000000180005e28     libiterobjreachobj004.obj
 0002:00000e60       ??_C@_0CA@EKPNJOEP@JVMTI_ERROR_UNSUPPORTED_VERSION@ 0000000180005e60     libiterobjreachobj004.obj
 0002:00000e80       ??_C@_0BN@OFFMAHHL@JVMTI_ERROR_NAMES_DONT_MATCH@ 0000000180005e80     libiterobjreachobj004.obj
 0002:00000ea0       ??_C@_0DN@HHBBLAKE@JVMTI_ERROR_UNSUPPORTED_REDEFIN@ 0000000180005ea0     libiterobjreachobj004.obj
 0002:00000ee0       ??_C@_0DO@HMBGBGNA@JVMTI_ERROR_UNSUPPORTED_REDEFIN@ 0000000180005ee0     libiterobjreachobj004.obj
 0002:00000f20       ??_C@_0BP@PBECGKHJ@JVMTI_ERROR_UNMODIFIABLE_CLASS@ 0000000180005f20     libiterobjreachobj004.obj
 0002:00000f40       ??_C@_0BK@CANILEHF@JVMTI_ERROR_NOT_AVAILABLE@ 0000000180005f40     libiterobjreachobj004.obj
 0002:00000f60       ??_C@_0CE@INJKMEFK@JVMTI_ERROR_MUST_POSSESS_CAPABI@ 0000000180005f60     libiterobjreachobj004.obj
 0002:00000f88       ??_C@_0BJ@LBFPFPDM@JVMTI_ERROR_NULL_POINTER@ 0000000180005f88     libiterobjreachobj004.obj
 0002:00000fa8       ??_C@_0BP@CHJPNNEM@JVMTI_ERROR_ABSENT_INFORMATION@ 0000000180005fa8     libiterobjreachobj004.obj
 0002:00000fc8       ??_C@_0BP@OMFMNLC@JVMTI_ERROR_INVALID_EVENT_TYPE@ 0000000180005fc8     libiterobjreachobj004.obj
 0002:00000fe8       ??_C@_0BN@BIBNPHHO@JVMTI_ERROR_ILLEGAL_ARGUMENT@ 0000000180005fe8     libiterobjreachobj004.obj
 0002:00001008       ??_C@_0BK@KKNDHDCE@JVMTI_ERROR_NATIVE_METHOD@ 0000000180006008     libiterobjreachobj004.obj
 0002:00001028       ??_C@_0BK@PMKCFHAE@JVMTI_ERROR_OUT_OF_MEMORY@ 0000000180006028     libiterobjreachobj004.obj
 0002:00001048       ??_C@_0BK@NNJBDMNB@JVMTI_ERROR_ACCESS_DENIED@ 0000000180006048     libiterobjreachobj004.obj
 0002:00001068       ??_C@_0BI@GHECLMNC@JVMTI_ERROR_WRONG_PHASE@ 0000000180006068     libiterobjreachobj004.obj
 0002:00001080       ??_C@_0BF@OLIHJOII@JVMTI_ERROR_INTERNAL@ 0000000180006080     libiterobjreachobj004.obj
 0002:00001098       ??_C@_0BO@EOHGKJHI@JVMTI_ERROR_UNATTACHED_THREAD@ 0000000180006098     libiterobjreachobj004.obj
 0002:000010b8       ??_C@_0CA@LKHFDACL@JVMTI_ERROR_INVALID_ENVIRONMENT@ 00000001800060b8     libiterobjreachobj004.obj
 0002:000010d8       ??_C@_0BA@MMFHLOKK@?$DMunknown?5error?$DO@ 00000001800060d8     libiterobjreachobj004.obj
 0002:000010e8       ??_C@_0CF@CBHOKDB@throwable?5?$DN?5jni?9?$DOExceptionOccur@ 00000001800060e8     libiterobjreachobj004.obj
 0002:00001110       ??_C@_03OFAPEBGM@?$CFs?6@  0000000180006110     libiterobjreachobj004.obj
 0002:00001118       ??_C@_0DM@LPIGEGNJ@s?2test?2hotspot?2jtreg?2vmTestbase@ 0000000180006118     libiterobjreachobj004.obj
 0002:00001158       ??_C@_0CC@NFCNPEPK@Exception?5in?5JNI?5call?5?$CIcleared?$CJ@ 0000000180006158     libiterobjreachobj004.obj
 0002:00001180       ??_C@_0BJ@IBAKFIKF@jni?9?$DOExceptionDescribe?$CI?$CJ@ 0000000180006180     libiterobjreachobj004.obj
 0002:000011a0       ??_C@_0BG@GGKALKMH@jni?9?$DOExceptionClear?$CI?$CJ@ 00000001800061a0     libiterobjreachobj004.obj
 0002:000011b8       ??_C@_0CF@JMGFGJLJ@?$CD?5?5?5verified?5JNI?5assertion?5is?5F@ 00000001800061b8     libiterobjreachobj004.obj
 0002:000011e0       ??_C@_07KBAMPNJK@verbose@  00000001800061e0     libiterobjreachobj004.obj
 0002:000011e8       ??_C@_0DN@PKJBOLAP@nsk_jvmti_parseOptions?$CI?$CJ?3?5unexp@ 00000001800061e8     libiterobjreachobj004.obj
 0002:00001228       ??_C@_05IMBNNINJ@trace@    0000000180006228     libiterobjreachobj004.obj
 0002:00001230       ??_C@_0DD@BJKGNDMB@nsk_jvmti_parseOptions?$CI?$CJ?3?5no?5va@ 0000000180006230     libiterobjreachobj004.obj
 0002:00001264       ??_C@_04CGFJFPFD@none@     0000000180006264     libiterobjreachobj004.obj
 0002:0000126c       ??_C@_06BMELKFMA@before@   000000018000626c     libiterobjreachobj004.obj
 0002:00001274       ??_C@_05CMKPCFDK@after@    0000000180006274     libiterobjreachobj004.obj
 0002:0000127c       ??_C@_03NFKEKGGK@all@      000000018000627c     libiterobjreachobj004.obj
 0002:00001280       ??_C@_0DM@NDNJGJKE@nsk_jvmti_parseOptions?$CI?$CJ?3?5uexpe@ 0000000180006280     libiterobjreachobj004.obj
 0002:000012c0       ??_C@_08NBBJKJO@waittime@  00000001800062c0     libiterobjreachobj004.obj
 0002:000012d0       ??_C@_0DO@CMHGAOHC@nsk_jvmti_parseOptions?$CI?$CJ?3?5not?5i@ 00000001800062d0     libiterobjreachobj004.obj
 0002:00001310       ??_C@_0DL@LNMPBDLN@nsk_jvmti_parseOptions?$CI?$CJ?3?5negat@ 0000000180006310     libiterobjreachobj004.obj
 0002:00001350       ??_C@_0DA@GMFJNOJH@nsk_jvmti_parseOptions?$CI?$CJ?3?5unkno@ 0000000180006350     libiterobjreachobj004.obj
 0002:00001380       ??_C@_0CO@CCIAMEAN@nsk_jvmti_parseOptions?$CI?$CJ?3?5found@ 0000000180006380     libiterobjreachobj004.obj
 0002:000013b0       ??_C@_0CJ@OEGPCGDL@nsk_jvmti_parseOptions?$CI?$CJ?3?5out?5o@ 00000001800063b0     libiterobjreachobj004.obj
 0002:000013e0       ??_C@_0DI@NMBHPGGF@nsk_jvmti_parseOptions?$CI?$CJ?3?5too?5m@ 00000001800063e0     libiterobjreachobj004.obj
 0002:00001418       ??_C@_03POGCGECB@?5?0?$HO@ 0000000180006418     libiterobjreachobj004.obj
 0002:00001420       ??_C@_0CB@MLNJNCLJ@?5?5jvmti?5error?3?5code?$DN?$CFd?0?5name?$DN?$CFs@ 0000000180006420     libiterobjreachobj004.obj
 0002:00001448       ??_C@_0CD@OHBGDKMK@?$CD?5?5?5jvmti?5error?3?5code?$DN?$CFd?0?5name?$DN@ 0000000180006448     libiterobjreachobj004.obj
 0002:00001470       ??_C@_0CG@JNNCGPHB@?$CD?5?5?5error?5expected?3?5code?$DN?$CFd?0?5na@ 0000000180006470     libiterobjreachobj004.obj
 0002:000014a0       ??_C@_0EB@IMGKPCGE@?$CIstr_obj?5?$DN?5jni?9?$DONewStringUTF?$CIco@ 00000001800064a0     libiterobjreachobj004.obj
 0002:000014f0       ??_C@_0EA@HFOGGBCC@s?2test?2hotspot?2jtreg?2vmTestbase@ 00000001800064f0     libiterobjreachobj004.obj
 0002:00001530       ??_C@_05KKCIMGE@error@     0000000180006530     libiterobjreachobj004.obj
 0002:00001538       ??_C@_0BD@HGNAOMCP@agent_data_monitor@ 0000000180006538     libiterobjreachobj004.obj
 0002:00001550       ??_C@_0EB@OGCLGKLN@javaVM?9?$DOGetEnv?$CI?$CIvoid?5?$CK?$CK?$CJ?$CGjvmti_@ 0000000180006550     libiterobjreachobj004.obj
 0002:000015a0       ??_C@_0EA@PNBCDMOA@s?2test?2hotspot?2jtreg?2vmTestbase@ 00000001800065a0     libiterobjreachobj004.obj
 0002:000015e0       ??_C@_0CI@DDPIFBGM@init_agent_data?$CIjvmti_env?0?5?$CGage@ 00000001800065e0     libiterobjreachobj004.obj
 0002:00001608       ??_C@_0DI@ILAHDLMP@?$CI?$CKagentThreadProc?$CJ?$CIjvmti_env?0?5a@ 0000000180006608     libiterobjreachobj004.obj
 0002:00001640       ??_C@_0BD@KDBALNLB@JVMTI?5agent?5thread@ 0000000180006640     libiterobjreachobj004.obj
 0002:00001658       ??_C@_0BB@NOKBFPFO@java?1lang?1Thread@ 0000000180006658     libiterobjreachobj004.obj
 0002:0000166c       ??_C@_06FALKBLGB@?$DMinit?$DO@ 000000018000666c     libiterobjreachobj004.obj
 0002:00001678       ??_C@_0BG@IKDDPPGD@?$CILjava?1lang?1String?$DL?$CJV@ 0000000180006678     libiterobjreachobj004.obj
 0002:00001690       ??_C@_0EB@IFJBFEKC@?$CIthreadClass?5?$DN?5jni_env?9?$DOFindCla@ 0000000180006690     libiterobjreachobj004.obj
 0002:000016e0       ??_C@_0GF@FGFIBKKL@?$CIthreadCtor?5?$DN?5jni_env?9?$DOGetMetho@ 00000001800066e0     libiterobjreachobj004.obj
 0002:00001748       ??_C@_0DN@NCPDJLOG@?$CIthreadName?5?$DN?5jni_env?9?$DONewStrin@ 0000000180006748     libiterobjreachobj004.obj
 0002:00001790       ??_C@_0FE@PFKODBGC@?$CIthreadObject?5?$DN?5jni_env?9?$DONewObj@ 0000000180006790     libiterobjreachobj004.obj
 0002:000017f0       ??_C@_0ED@HOBAHHJI@?$CIthreadGlobalRef?5?$DN?5jni_env?9?$DONew@ 00000001800067f0     libiterobjreachobj004.obj
 0002:00001840       ??_C@_0FN@HNJJAHFC@jvmti_env?9?$DORunAgentThread?$CIagent@ 0000000180006840     libiterobjreachobj004.obj
 0002:000018a0       ??_C@_0EA@MOJDNKDF@Debuggee?5status?5sync?5aborted?5be@ 00000001800068a0     libiterobjreachobj004.obj
 0002:000018e0       ??_C@_0CO@PGPGMHBJ@No?5status?5sync?5occured?5for?5time@ 00000001800068e0     libiterobjreachobj004.obj
 0002:00001910       ??_C@_0CL@DOEBDPKJ@Debuggee?5was?5not?5suspended?5on?5s@ 0000000180006910     libiterobjreachobj004.obj
 0002:00001940       ??_C@_0EA@EEOEJAEN@status?5?$DN?5syncDebuggeeStatus?$CIjni@ 0000000180006940     libiterobjreachobj004.obj
 0002:00001980       ??_C@_0BL@JBCFNBMB@nsk_jvmti_resetAgentData?$CI?$CJ@ 0000000180006980     libiterobjreachobj004.obj
 0002:000019a0       ??_C@_0BF@KACGOIM@signature?5?$CB?$DN?5nullptr@ 00000001800069a0     libiterobjreachobj004.obj
 0002:000019b8       ??_C@_0CO@PPMOIPJN@jvmti_env?9?$DOGetLoadedClasses?$CI?$CGco@ 00000001800069b8     libiterobjreachobj004.obj
 0002:000019e8       ??_C@_0DJ@MPPHCAIG@jvmti_env?9?$DOGetClassSignature?$CIcl@ 00000001800069e8     libiterobjreachobj004.obj
 0002:00001a28       ??_C@_0CL@KGBLFGIP@jvmti_env?9?$DODeallocate?$CI?$CIunsigned@ 0000000180006a28     libiterobjreachobj004.obj
 0002:00001a58       ??_C@_0CP@MLOCFBGK@jvmti_env?9?$DODeallocate?$CI?$CIunsigned@ 0000000180006a58     libiterobjreachobj004.obj
 0002:00001a88       ??_C@_0CP@MBBGLPFK@jvmti_env?9?$DODeallocate?$CI?$CIunsigned@ 0000000180006a88     libiterobjreachobj004.obj
 0002:00001ac0       ??_C@_0EF@HIEPFNJF@?$CIfoundClass?5?$DN?5?$CIjclass?$CJ?5jni_env?9@ 0000000180006ac0     libiterobjreachobj004.obj
 0002:00001b10       ??_C@_0EL@LPBEELIP@s?2test?2hotspot?2jtreg?2vmTestbase@ 0000000180006b10     libiterobjreachobj004.obj
 0002:00001b60       ??_C@_0CK@JDAMFDMJ@jvmti?9?$DOSetTag?$CIo?0?5tag?$CJ?5?$DN?$DN?5JVMTI_@ 0000000180006b60     libiterobjreachobj004.obj
 0002:00001b90       ??_C@_0CC@DAMNHKNI@Can?8t?5set?5tag?5?$CFli?5for?5object?5?$CFl@ 0000000180006b90     libiterobjreachobj004.obj
 0002:00001bb8       ??_C@_0DL@HAJPNKEF@jvmti?9?$DOGetObjectHashCode?$CIo?0?5?$CGha@ 0000000180006bb8     libiterobjreachobj004.obj
 0002:00001bf8       ??_C@_0BL@JFPIEOBF@Can?8t?5get?5hash?5object?5?$CFlx?6@ 0000000180006bf8     libiterobjreachobj004.obj
 0002:00001c18       ??_C@_0BG@DICPHBKN@setTag?3?5?$CF08x?5?$DM?9?5?$CF?53li@ 0000000180006c18     libiterobjreachobj004.obj
 0002:00001c30       ??_C@_0DH@FCEEBDMJ@?$CIs?5?$DN?5jni?9?$DOGetStringUTFChars?$CIsIn@ 0000000180006c30     libiterobjreachobj004.obj
 0002:00001c68       ??_C@_0BJ@OKKGHDCN@Can?8t?5get?5string?5at?5?$CF?$CDp?6@ 0000000180006c68     libiterobjreachobj004.obj
 0002:00001c88       ??_C@_0BP@EKFLGGFJ@Can?8t?5get?5string?5at?5?$CF?$CDp?3?5null?6@ 0000000180006c88     libiterobjreachobj004.obj
 0002:00001ca8       ??_C@_06ICODBHCL@?5?1?1?5?$CFs@ 0000000180006ca8     libiterobjreachobj004.obj
 0002:00001cb0       ??_C@_0DB@KGFPLEGO@?$CIr?5?$DN?5jvmti?9?$DOGetTag?$CIo?0?5?$CGtag?$CJ?$CJ?5?$DN?$DN@ 0000000180006cb0     libiterobjreachobj004.obj
 0002:00001ce8       ??_C@_0CO@PDAGBCGJ@Can?8t?5GetTag?5for?5object?5?$CFlx?4?5Re@ 0000000180006ce8     libiterobjreachobj004.obj
 0002:00001d18       ??_C@_0CH@HPEODOHC@TEST_BUG?3?5Max?4?5number?5of?5refs?5r@ 0000000180006d18     libiterobjreachobj004.obj
 0002:00001d40       ??_C@_0DI@PHFCABIM@?$CIr?5?$DN?5jvmti?9?$DOGetTag?$CIfrom?0?5?$CGtagFr@ 0000000180006d40     libiterobjreachobj004.obj
 0002:00001d78       ??_C@_0DI@MDEGFNKD@TEST_BUG?3?5Can?8t?5GetTag?5for?5obje@ 0000000180006d78     libiterobjreachobj004.obj
 0002:00001db0       ??_C@_0DE@MLELJAHM@?$CIr?5?$DN?5jvmti?9?$DOGetTag?$CIto?0?5?$CGtagTo?$CJ?$CJ@ 0000000180006db0     libiterobjreachobj004.obj
 0002:00001de8       ??_C@_0DD@LENNLEMO@st_jvmti?9?$DOSetEnvironmentLocalSt@ 0000000180006de8     libiterobjreachobj004.obj
 0002:00001e20       ??_C@_0HK@JCNHADLH@s?2test?2hotspot?2jtreg?2vmTestbase@ 0000000180006e20     libiterobjreachobj004.obj
 0002:00001ea0       ??_C@_0DD@OCELELDD@st_jvmti?9?$DOGetEnvironmentLocalSt@ 0000000180006ea0     libiterobjreachobj004.obj
 0002:00001ed8       ??_C@_0BI@BGHFFELJ@Wait?5for?5debugee?5start?6@ 0000000180006ed8     libiterobjreachobj004.obj
 0002:00001ef0       ??_C@_0BP@LAIJOMPC@nsk_jvmti_waitForSync?$CItimeout?$CJ@ 0000000180006ef0     libiterobjreachobj004.obj
 0002:00001f10       ??_C@_0BI@ENEOJHP@Find?5debugee?5class?3?5?$CFs?6@ 0000000180006f10     libiterobjreachobj004.obj
 0002:00001f28       ??_C@_0CI@IPDCJCKO@Find?5static?5field?5in?5debugee?5cl@ 0000000180006f28     libiterobjreachobj004.obj
 0002:00001f50       ??_C@_0GI@CFHEFDEO@?$CIobjectField?5?$DN?5jni?9?$DOGetStaticFi@ 0000000180006f50     libiterobjreachobj004.obj
 0002:00001fb8       ??_C@_0DB@PCCDMNK@Find?5value?5of?5static?5field?5in?5d@ 0000000180006fb8     libiterobjreachobj004.obj
 0002:00001ff0       ??_C@_0EL@FFNBNLCG@?$CIobject?5?$DN?5jni?9?$DOGetStaticObjectF@ 0000000180006ff0     libiterobjreachobj004.obj
 0002:00002040       ??_C@_0FE@POGHAFHB@Calling?5IterateOverObjectsReach@ 0000000180007040     libiterobjreachobj004.obj
 0002:000020a0       ??_C@_0FO@BBOJJDAP@jvmti?9?$DOIterateOverObjectsReacha@ 00000001800070a0     libiterobjreachobj004.obj
 0002:00002100       ??_C@_0EH@JLDCIOBP@IterateOverObjectsReachableFrom@ 0000000180007100     libiterobjreachobj004.obj
 0002:00002148       ??_C@_0DP@FAOBABGD@Local?5storage?5address?5was?5corru@ 0000000180007148     libiterobjreachobj004.obj
 0002:00002188       ??_C@_0DH@PGIJIGKG@Local?5storage?5was?5corrupted?3?5?$CFs@ 0000000180007188     libiterobjreachobj004.obj
 0002:000021c0       ??_C@_0BH@HPEOJMHL@Let?5debugee?5to?5finish?6@ 00000001800071c0     libiterobjreachobj004.obj
 0002:000021d8       ??_C@_0BH@LECMGIIA@nsk_jvmti_resumeSync?$CI?$CJ@ 00000001800071d8     libiterobjreachobj004.obj
 0002:000021f0       ??_C@_0CA@MNKGCBCG@nsk_jvmti_parseOptions?$CIoptions?$CJ@ 00000001800071f0     libiterobjreachobj004.obj
 0002:00002210       ??_C@_0DN@MIAMNFPH@?$CIjvmti?5?$DN?5nsk_jvmti_createJVMTIE@ 0000000180007210     libiterobjreachobj004.obj
 0002:00002250       ??_C@_0BO@DBKDIPGD@jvmti?9?$DOAddCapabilities?$CI?$CGcaps?$CJ@ 0000000180007250     libiterobjreachobj004.obj
 0002:00002270       ??_C@_0CL@PIACJIPK@nsk_jvmti_setAgentProc?$CIagentPro@ 0000000180007270     libiterobjreachobj004.obj
 0002:000022b0       ??_C@_1EC@JIJBPKFM@?$AAa?$AAp?$AAi?$AA?9?$AAm?$AAs?$AA?9?$AAw?$AAi?$AAn?$AA?9?$AAc?$AAo?$AAr?$AAe@ 00000001800072b0     MSVCRT:thread_safe_statics.obj
 0002:000022f8       ??_C@_1BK@MGMFAEKH@?$AAk?$AAe?$AAr?$AAn?$AAe?$AAl?$AA3?$AA2?$AA?4?$AAd?$AAl?$AAl@ 00000001800072f8     MSVCRT:thread_safe_statics.obj
 0002:00002318       ??_C@_0BJ@JEBJOJFJ@SleepConditionVariableCS@ 0000000180007318     MSVCRT:thread_safe_statics.obj
 0002:00002338       ??_C@_0BJ@PGPPEPCC@WakeAllConditionVariable@ 0000000180007338     MSVCRT:thread_safe_statics.obj
 0002:00002358       _pDefaultRawDllMain        0000000180007358     MSVCRT:dll_dllmain.obj
 0002:00002358       _pRawDllMain               0000000180007358     MSVCRT:dll_dllmain.obj
 0002:00002360       __xmm@ffffffffffffffffffffffffffffffff 0000000180007360     MSVCRT:utility.obj
 0002:00002370       _load_config_used          0000000180007370     MSVCRT:loadcfg.obj
 0002:00002580       _tls_used                  0000000180007580     MSVCRT:tlssup.obj
 0002:000025a8       __volatile_metadata        00000001800075a8     <linker-defined>
 0002:000029c0       __rtc_iaa                  00000001800079c0     MSVCRT:initsect.obj
 0002:000029c8       __rtc_izz                  00000001800079c8     MSVCRT:initsect.obj
 0002:000029d0       __rtc_taa                  00000001800079d0     MSVCRT:initsect.obj
 0002:000029d8       __rtc_tzz                  00000001800079d8     MSVCRT:initsect.obj
 0002:000029e0       _tls_start                 00000001800079e0     MSVCRT:tlssup.obj
 0002:000029e4       _Init_thread_epoch         00000001800079e4     MSVCRT:thread_safe_statics.obj
 0002:000029e8       _tls_end                   00000001800079e8     MSVCRT:tlssup.obj
 0002:0000309c       __IMPORT_DESCRIPTOR_KERNEL32 000000018000809c     kernel32:KERNEL32.dll
 0002:000030b0       __IMPORT_DESCRIPTOR_VCRUNTIME140 00000001800080b0     vcruntime:VCRUNTIME140.dll
 0002:000030c4       __IMPORT_DESCRIPTOR_api-ms-win-crt-heap-l1-1-0 00000001800080c4     ucrt:api-ms-win-crt-heap-l1-1-0.dll
 0002:000030d8       __IMPORT_DESCRIPTOR_api-ms-win-crt-runtime-l1-1-0 00000001800080d8     ucrt:api-ms-win-crt-runtime-l1-1-0.dll
 0002:000030ec       __IMPORT_DESCRIPTOR_api-ms-win-crt-convert-l1-1-0 00000001800080ec     ucrt:api-ms-win-crt-convert-l1-1-0.dll
 0002:00003100       __IMPORT_DESCRIPTOR_api-ms-win-crt-stdio-l1-1-0 0000000180008100     ucrt:api-ms-win-crt-stdio-l1-1-0.dll
 0002:00003114       __IMPORT_DESCRIPTOR_api-ms-win-crt-string-l1-1-0 0000000180008114     ucrt:api-ms-win-crt-string-l1-1-0.dll
 0002:00003128       __NULL_IMPORT_DESCRIPTOR   0000000180008128     kernel32:KERNEL32.dll
 0003:00000048       _Init_global_epoch         0000000180009048     MSVCRT:thread_safe_statics.obj
 0003:00000050       __security_cookie          0000000180009050     MSVCRT:gs_cookie.obj
 0003:00000058       __security_cookie_complement 0000000180009058     MSVCRT:gs_cookie.obj
 0003:00000060       __scrt_native_dllmain_reason 0000000180009060     MSVCRT:utility.obj
 0003:00000068       __isa_available            0000000180009068     MSVCRT:cpu_disp.obj
 0003:0000006c       __isa_enabled              000000018000906c     MSVCRT:cpu_disp.obj
 0003:00000070       __memset_fast_string_threshold 0000000180009070     MSVCRT:cpu_disp.obj
 0003:00000078       __memset_nt_threshold      0000000180009078     MSVCRT:cpu_disp.obj
 0003:00000080       __scrt_ucrt_dll_is_in_use  0000000180009080     MSVCRT:ucrt_stubs.obj
 0003:00000090       g_wrongHeapCallbacks       0000000180009090     libiterobjreachobj004.obj
 0003:00000110       g_szTagInfo                0000000180009110     libiterobjreachobj004.obj
 0003:00002050       g_tagFlags                 000000018000b050     libiterobjreachobj004.obj
 0003:00002438       g_refsToVerifyCnt          000000018000b438     libiterobjreachobj004.obj
 0003:0000243c       g_fakeUserData             000000018000b43c     libiterobjreachobj004.obj
 0003:00002440       g_tagVisitCount            000000018000b440     libiterobjreachobj004.obj
 0003:000033e0       g_refsToVerify             000000018000c3e0     libiterobjreachobj004.obj
 0003:0001aae0       g_userDataError            0000000180023ae0     libiterobjreachobj004.obj
 0003:0001ac98       ?_OptionsStorage@?1??__local_stdio_printf_options@@9@4_KA 0000000180023c98     libiterobjreachobj004.obj
 0003:0001b258       _tls_index                 0000000180024258     MSVCRT:tlssup.obj
 0003:0001b260       __scrt_current_native_startup_state 0000000180024260     MSVCRT:utility.obj
 0003:0001b268       __scrt_native_startup_lock 0000000180024268     MSVCRT:utility.obj
 0003:0001b2a8       __scrt_debugger_hook_flag  00000001800242a8     MSVCRT:utility_desktop.obj
 0003:0001b2b0       ?__type_info_root_node@@3U__type_info_node@@A 00000001800242b0     MSVCRT:tncleanup.obj
 0003:0001b2c0       ?_OptionsStorage@?1??__local_stdio_scanf_options@@9@4_KA 00000001800242c0     MSVCRT:default_local_stdio_options.obj
 0003:0001b2c8       __favor                    00000001800242c8     MSVCRT:cpu_disp.obj
 0003:0001b2d0       __dyn_tls_init_callback    00000001800242d0     <common>

 entry point at        0001:000030f0

 Static symbols

 0000:fffd9000       .debug$S                   0000000180000000     iterobjreachobj004.exp
 0000:fffd9000       .debug$S                   0000000180000000     vcruntime:VCRUNTIME140.dll
 0000:fffd9000       .debug$S                   0000000180000000     vcruntime:VCRUNTIME140.dll
 0000:fffd9000       .debug$S                   0000000180000000     vcruntime:VCRUNTIME140.dll
 0000:fffd9000       .debug$S                   0000000180000000     vcruntime:VCRUNTIME140.dll
 0000:fffd9000       .debug$S                   0000000180000000     vcruntime:VCRUNTIME140.dll
 0000:fffd9000       .debug$S                   0000000180000000     vcruntime:VCRUNTIME140.dll
 0000:fffd9000       .debug$S                   0000000180000000     vcruntime:VCRUNTIME140.dll
 0000:fffd9000       .debug$S                   0000000180000000     ucrt:api-ms-win-crt-convert-l1-1-0.dll
 0000:fffd9000       .debug$S                   0000000180000000     ucrt:api-ms-win-crt-heap-l1-1-0.dll
 0000:fffd9000       .debug$S                   0000000180000000     ucrt:api-ms-win-crt-heap-l1-1-0.dll
 0000:fffd9000       .debug$S                   0000000180000000     ucrt:api-ms-win-crt-heap-l1-1-0.dll
 0000:fffd9000       .debug$S                   0000000180000000     ucrt:api-ms-win-crt-heap-l1-1-0.dll
 0000:fffd9000       .debug$S                   0000000180000000     ucrt:api-ms-win-crt-runtime-l1-1-0.dll
 0000:fffd9000       .debug$S                   0000000180000000     ucrt:api-ms-win-crt-runtime-l1-1-0.dll
 0000:fffd9000       .debug$S                   0000000180000000     ucrt:api-ms-win-crt-runtime-l1-1-0.dll
 0000:fffd9000       .debug$S                   0000000180000000     ucrt:api-ms-win-crt-runtime-l1-1-0.dll
 0000:fffd9000       .debug$S                   0000000180000000     ucrt:api-ms-win-crt-runtime-l1-1-0.dll
 0000:fffd9000       .debug$S                   0000000180000000     ucrt:api-ms-win-crt-runtime-l1-1-0.dll
 0000:fffd9000       .debug$S                   0000000180000000     ucrt:api-ms-win-crt-runtime-l1-1-0.dll
 0000:fffd9000       .debug$S                   0000000180000000     ucrt:api-ms-win-crt-runtime-l1-1-0.dll
 0000:fffd9000       .debug$S                   0000000180000000     ucrt:api-ms-win-crt-runtime-l1-1-0.dll
 0000:fffd9000       .debug$S                   0000000180000000     ucrt:api-ms-win-crt-runtime-l1-1-0.dll
 0000:fffd9000       .debug$S                   0000000180000000     ucrt:api-ms-win-crt-runtime-l1-1-0.dll
 0000:fffd9000       .debug$S                   0000000180000000     ucrt:api-ms-win-crt-runtime-l1-1-0.dll
 0000:fffd9000       .debug$S                   0000000180000000     ucrt:api-ms-win-crt-runtime-l1-1-0.dll
 0000:fffd9000       .debug$S                   0000000180000000     ucrt:api-ms-win-crt-runtime-l1-1-0.dll
 0000:fffd9000       .debug$S                   0000000180000000     ucrt:api-ms-win-crt-runtime-l1-1-0.dll
 0000:fffd9000       .debug$S                   0000000180000000     ucrt:api-ms-win-crt-runtime-l1-1-0.dll
 0000:fffd9000       .debug$S                   0000000180000000     ucrt:api-ms-win-crt-stdio-l1-1-0.dll
 0000:fffd9000       .debug$S                   0000000180000000     ucrt:api-ms-win-crt-stdio-l1-1-0.dll
 0000:fffd9000       .debug$S                   0000000180000000     ucrt:api-ms-win-crt-stdio-l1-1-0.dll
 0000:fffd9000       .debug$S                   0000000180000000     ucrt:api-ms-win-crt-stdio-l1-1-0.dll
 0000:fffd9000       .debug$S                   0000000180000000     ucrt:api-ms-win-crt-stdio-l1-1-0.dll
 0000:fffd9000       .debug$S                   0000000180000000     ucrt:api-ms-win-crt-stdio-l1-1-0.dll
 0000:fffd9000       .debug$S                   0000000180000000     ucrt:api-ms-win-crt-stdio-l1-1-0.dll
 0000:fffd9000       .debug$S                   0000000180000000     ucrt:api-ms-win-crt-stdio-l1-1-0.dll
 0000:fffd9000       .debug$S                   0000000180000000     ucrt:api-ms-win-crt-stdio-l1-1-0.dll
 0000:fffd9000       .debug$S                   0000000180000000     ucrt:api-ms-win-crt-stdio-l1-1-0.dll
 0000:fffd9000       .debug$S                   0000000180000000     ucrt:api-ms-win-crt-string-l1-1-0.dll
 0000:fffd9000       .debug$S                   0000000180000000     ucrt:api-ms-win-crt-string-l1-1-0.dll
 0000:fffd9000       .debug$S                   0000000180000000     ucrt:api-ms-win-crt-string-l1-1-0.dll
 0000:fffd9000       .debug$S                   0000000180000000     ucrt:api-ms-win-crt-string-l1-1-0.dll
 0000:fffd9000       .debug$S                   0000000180000000     ucrt:api-ms-win-crt-string-l1-1-0.dll
 0000:fffd9000       .debug$S                   0000000180000000     ucrt:api-ms-win-crt-string-l1-1-0.dll
 0000:fffd9000       .debug$S                   0000000180000000     ucrt:api-ms-win-crt-string-l1-1-0.dll
 0000:fffd9000       .debug$S                   0000000180000000     ucrt:api-ms-win-crt-string-l1-1-0.dll
 0000:fffd9000       .debug$S                   0000000180000000     kernel32:KERNEL32.dll
 0000:fffd9000       .debug$S                   0000000180000000     kernel32:KERNEL32.dll
 0000:fffd9000       .debug$S                   0000000180000000     kernel32:KERNEL32.dll
 0000:fffd9000       .debug$S                   0000000180000000     kernel32:KERNEL32.dll
 0000:fffd9000       .debug$S                   0000000180000000     kernel32:KERNEL32.dll
 0000:fffd9000       .debug$S                   0000000180000000     kernel32:KERNEL32.dll
 0000:fffd9000       .debug$S                   0000000180000000     kernel32:KERNEL32.dll
 0000:fffd9000       .debug$S                   0000000180000000     kernel32:KERNEL32.dll
 0000:fffd9000       .debug$S                   0000000180000000     kernel32:KERNEL32.dll
 0000:fffd9000       .debug$S                   0000000180000000     kernel32:KERNEL32.dll
 0000:fffd9000       .debug$S                   0000000180000000     kernel32:KERNEL32.dll
 0000:fffd9000       .debug$S                   0000000180000000     kernel32:KERNEL32.dll
 0000:fffd9000       .debug$S                   0000000180000000     kernel32:KERNEL32.dll
 0000:fffd9000       .debug$S                   0000000180000000     kernel32:KERNEL32.dll
 0000:fffd9000       .debug$S                   0000000180000000     kernel32:KERNEL32.dll
 0000:fffd9000       .debug$S                   0000000180000000     kernel32:KERNEL32.dll
 0000:fffd9000       .debug$S                   0000000180000000     kernel32:KERNEL32.dll
 0000:fffd9000       .debug$S                   0000000180000000     kernel32:KERNEL32.dll
 0000:fffd9000       .debug$S                   0000000180000000     kernel32:KERNEL32.dll
 0000:fffd9000       .debug$S                   0000000180000000     kernel32:KERNEL32.dll
 0000:fffd9000       .debug$S                   0000000180000000     kernel32:KERNEL32.dll
 0000:fffd9000       .debug$S                   0000000180000000     kernel32:KERNEL32.dll
 0000:fffd9000       .debug$S                   0000000180000000     kernel32:KERNEL32.dll
 0000:fffd9000       .debug$S                   0000000180000000     kernel32:KERNEL32.dll
 0000:fffd9000       .debug$S                   0000000180000000     kernel32:KERNEL32.dll
 0000:fffd9000       .debug$S                   0000000180000000     kernel32:KERNEL32.dll
 0000:fffd9000       .debug$S                   0000000180000000     kernel32:KERNEL32.dll
 0000:fffd9000       .debug$S                   0000000180000000     kernel32:KERNEL32.dll
 0001:00000e18       addRefToVerify             0000000180001e18 f   libiterobjreachobj004.obj
 0001:00000e8c       agentProc                  0000000180001e8c f   libiterobjreachobj004.obj
 0001:00001224       agentThreadWrapper         0000000180002224 f   libiterobjreachobj004.obj
 0001:00001378       check_option               0000000180002378 f   libiterobjreachobj004.obj
 0001:000015c0       file_basename              00000001800025c0 f   libiterobjreachobj004.obj
 0001:000025f8       startAgentThreadWrapper    00000001800035f8 f   libiterobjreachobj004.obj
 0001:00002924       syncDebuggeeStatus         0000000180003924 f   libiterobjreachobj004.obj
 0001:00002bac       capture_previous_context   0000000180003bac f   MSVCRT:gs_report.obj
 0001:00002c20       ?__scrt_initialize_thread_safe_statics@@YAHXZ 0000000180003c20 f   MSVCRT:thread_safe_statics.obj
 0001:00002cf0       ?__scrt_uninitialize_thread_safe_statics@@YAXXZ 0000000180003cf0 f   MSVCRT:thread_safe_statics.obj
 0001:00002da0       $$000000                   0000000180003da0     MSVCRT:amdsecgs.obj
 0001:00002dd0       ?dllmain_crt_dispatch@@YAHQEAUHINSTANCE__@@KQEAX@Z 0000000180003dd0 f   MSVCRT:dll_dllmain.obj
 0001:00002e20       ?dllmain_crt_process_attach@@YAHQEAUHINSTANCE__@@QEAX@Z 0000000180003e20 f   MSVCRT:dll_dllmain.obj
 0001:00002f38       ?dllmain_crt_process_detach@@YAH_N@Z 0000000180003f38 f   MSVCRT:dll_dllmain.obj
 0001:00002fbc       ?dllmain_dispatch@@YAHQEAUHINSTANCE__@@KQEAX@Z 0000000180003fbc f   MSVCRT:dll_dllmain.obj
 0001:000039d0       $$000000                   00000001800049d0     MSVCRT:guard_dispatch.obj
 0001:000039f0       $$000000                   00000001800049f0     MSVCRT:guard_xfg_dispatch.obj
 0001:00003a06       ?fin$0@?0??dllmain_crt_process_attach@@YAHQEAUHINSTANCE__@@QEAX@Z@4HA 0000000180004a06 f   MSVCRT:dll_dllmain.obj
 0001:00003a1d       ?fin$0@?0??dllmain_crt_process_detach@@YAH_N@Z@4HA 0000000180004a1d f   MSVCRT:dll_dllmain.obj
 0001:00003a36       ?fin$1@?0??dllmain_crt_process_detach@@YAH_N@Z@4HA 0000000180004a36 f   MSVCRT:dll_dllmain.obj
 0001:00003a4a       ?filt$0@?0??dllmain_dispatch@@YAHQEAUHINSTANCE__@@KQEAX@Z@4HA 0000000180004a4a f   MSVCRT:dll_dllmain.obj
 0001:00003a80       __scrt_is_nonwritable_in_current_image$filt$0 0000000180004a80 f   MSVCRT:utility.obj
 0002:00000218       ?__scrt_initialize_tss_var@@3P6AHXZEA 0000000180005218     MSVCRT:thread_safe_statics.obj
 0002:00000340       ?opcLengths@@3QBEB         0000000180005340     libiterobjreachobj004.obj
 0002:000022a0       GS_ExceptionPointers       00000001800072a0     MSVCRT:gs_report.obj
 0002:000029f0       $unwind$fprintf            00000001800079f0     libiterobjreachobj004.obj
 0002:000029fc       $unwind$printf             00000001800079fc     libiterobjreachobj004.obj
 0002:00002a08       $unwind$?NewObject@JNIEnv_@@QEAAPEAV_jobject@@PEAV_jclass@@PEAU_jmethodID@@ZZ 0000000180007a08     libiterobjreachobj004.obj
 0002:00002a08       $unwind$nsk_lcomplain      0000000180007a08     libiterobjreachobj004.obj
 0002:00002a08       $unwind$nsk_ldisplay       0000000180007a08     libiterobjreachobj004.obj
 0002:00002a10       $unwind$nsk_lvdisplay      0000000180007a10     libiterobjreachobj004.obj
 0002:00002a10       $unwind$_RTC_Initialize    0000000180007a10     MSVCRT:initsect.obj
 0002:00002a10       $unwind$_RTC_Terminate     0000000180007a10     MSVCRT:initsect.obj
 0002:00002a10       $unwind$?__scrt_initialize_thread_safe_statics@@YAHXZ 0000000180007a10     MSVCRT:thread_safe_statics.obj
 0002:00002a1c       $unwind$nsk_complain       0000000180007a1c     libiterobjreachobj004.obj
 0002:00002a1c       $unwind$nsk_printf         0000000180007a1c     libiterobjreachobj004.obj
 0002:00002a24       $unwind$nsk_lvcomplain     0000000180007a24     libiterobjreachobj004.obj
 0002:00002a3c       $unwind$nsk_ltrace         0000000180007a3c     libiterobjreachobj004.obj
 0002:00002a3c       $unwind$__report_gsfailure 0000000180007a3c     MSVCRT:gs_report.obj
 0002:00002a44       $unwind$nsk_lvtrace        0000000180007a44     libiterobjreachobj004.obj
 0002:00002a44       $unwind$__raise_securityfailure 0000000180007a44     MSVCRT:gs_report.obj
 0002:00002a44       $unwind$__scrt_initialize_crt 0000000180007a44     MSVCRT:utility.obj
 0002:00002a44       $unwind$__scrt_initialize_onexit_tables 0000000180007a44     MSVCRT:utility.obj
 0002:00002a44       $unwind$__scrt_release_startup_lock 0000000180007a44     MSVCRT:utility.obj
 0002:00002a44       $unwind$__scrt_uninitialize_crt 0000000180007a44     MSVCRT:utility.obj
 0002:00002a44       $unwind$_onexit            0000000180007a44     MSVCRT:utility.obj
 0002:00002a4c       $unwind$nsk_lverify        0000000180007a4c     libiterobjreachobj004.obj
 0002:00002a5c       $unwind$nsk_vprintf        0000000180007a5c     libiterobjreachobj004.obj
 0002:00002a6c       $unwind$?nsk_jni_lverify@@YAHHPEAUJNIEnv_@@HQEBDH1ZZ 0000000180007a6c     libiterobjreachobj004.obj
 0002:00002a80       $unwind$?nsk_jni_check_exception@@YAHPEAUJNIEnv_@@QEBDH@Z 0000000180007a80     libiterobjreachobj004.obj
 0002:00002a9c       $unwind$nsk_jvmti_parseOptions 0000000180007a9c     libiterobjreachobj004.obj
 0002:00002ab8       $unwind$nsk_jvmti_createJVMTIEnv 0000000180007ab8     libiterobjreachobj004.obj
 0002:00002acc       $unwind$check_option       0000000180007acc     libiterobjreachobj004.obj
 0002:00002acc       $unwind$nsk_jvmti_waitForSync 0000000180007acc     libiterobjreachobj004.obj
 0002:00002acc       $unwind$_DllMainCRTStartup 0000000180007acc     MSVCRT:dll_dllmain.obj
 0002:00002adc       $unwind$Java_nsk_jvmti_unit_FollowReferences_FollowRefObjects_resetTags 0000000180007adc     libiterobjreachobj004.obj
 0002:00002adc       $unwind$addRefToVerify     0000000180007adc     libiterobjreachobj004.obj
 0002:00002adc       $unwind$nsk_jvmti_resetAgentData 0000000180007adc     libiterobjreachobj004.obj
 0002:00002adc       $unwind$nsk_jvmti_resumeSync 0000000180007adc     libiterobjreachobj004.obj
 0002:00002adc       $unwind$__scrt_initialize_default_local_stdio_options 0000000180007adc     MSVCRT:default_local_stdio_options.obj
 0002:00002adc       $unwind$?dllmain_crt_dispatch@@YAHQEAUHINSTANCE__@@KQEAX@Z 0000000180007adc     MSVCRT:dll_dllmain.obj
 0002:00002adc       $unwind$DllMain            0000000180007adc     MSVCRT:dll_dllmain_stub.obj
 0002:00002adc       $unwind$__GSHandlerCheck   0000000180007adc     MSVCRT:gshandler.obj
 0002:00002adc       $unwind$?__scrt_uninitialize_thread_safe_statics@@YAXXZ 0000000180007adc     MSVCRT:thread_safe_statics.obj
 0002:00002adc       $unwind$__scrt_acquire_startup_lock 0000000180007adc     MSVCRT:utility.obj
 0002:00002adc       $unwind$__scrt_dllmain_after_initialize_c 0000000180007adc     MSVCRT:utility.obj
 0002:00002adc       $unwind$__scrt_dllmain_before_initialize_c 0000000180007adc     MSVCRT:utility.obj
 0002:00002adc       $unwind$__scrt_dllmain_crt_thread_attach 0000000180007adc     MSVCRT:utility.obj
 0002:00002adc       $unwind$__scrt_dllmain_crt_thread_detach 0000000180007adc     MSVCRT:utility.obj
 0002:00002adc       $unwind$__scrt_dllmain_uninitialize_c 0000000180007adc     MSVCRT:utility.obj
 0002:00002adc       $unwind$__scrt_dllmain_uninitialize_critical 0000000180007adc     MSVCRT:utility.obj
 0002:00002adc       $unwind$atexit             0000000180007adc     MSVCRT:utility.obj
 0002:00002ae4       $unwind$nsk_jvmti_classBySignature 0000000180007ae4     libiterobjreachobj004.obj
 0002:00002af8       $unwind$nsk_jvmti_lverify  0000000180007af8     libiterobjreachobj004.obj
 0002:00002b0c       $unwind$exitOnError        0000000180007b0c     libiterobjreachobj004.obj
 0002:00002b1c       $unwind$Java_nsk_share_jvmti_ArgumentHandler_getAgentOptionsString 0000000180007b1c     libiterobjreachobj004.obj
 0002:00002b30       $unwind$Java_nsk_jvmti_unit_FollowReferences_FollowRefObjects_getTag 0000000180007b30     libiterobjreachobj004.obj
 0002:00002b30       $unwind$Java_nsk_share_jvmti_DebugeeClass_checkStatus 0000000180007b30     libiterobjreachobj004.obj
 0002:00002b30       $unwind$agentThreadWrapper 0000000180007b30     libiterobjreachobj004.obj
 0002:00002b40       $unwind$agentProc          0000000180007b40     libiterobjreachobj004.obj
 0002:00002b40       $unwind$startAgentThreadWrapper 0000000180007b40     libiterobjreachobj004.obj
 0002:00002b5c       $unwind$syncDebuggeeStatus 0000000180007b5c     libiterobjreachobj004.obj
 0002:00002b5c       $unwind$__scrt_dllmain_exception_filter 0000000180007b5c     MSVCRT:utility.obj
 0002:00002b70       $unwind$Java_nsk_share_jvmti_DebugeeClass_resetAgentData 0000000180007b70     libiterobjreachobj004.obj
 0002:00002b78       $unwind$MA_checkStatus     0000000180007b78     libiterobjreachobj004.obj
 0002:00002b8c       $unwind$Java_nsk_jvmti_unit_FollowReferences_FollowRefObjects_setTag 0000000180007b8c     libiterobjreachobj004.obj
 0002:00002ba4       $unwind$Java_nsk_jvmti_unit_FollowReferences_FollowRefObjects_addRefToVerify 0000000180007ba4     libiterobjreachobj004.obj
 0002:00002bc0       $unwind$Agent_Initialize   0000000180007bc0     libiterobjreachobj004.obj
 0002:00002bdc       $unwind$objectReferenceCallback 0000000180007bdc     libiterobjreachobj004.obj
 0002:00002be8       $unwind$capture_previous_context 0000000180007be8     MSVCRT:gs_report.obj
 0002:00002bf4       $unwind$__GSHandlerCheckCommon 0000000180007bf4     MSVCRT:gshandler.obj
 0002:00002c00       $xdatasym                  0000000180007c00     MSVCRT:amdsecgs.obj
 0002:00002c04       $unwind$?dllmain_crt_process_attach@@YAHQEAUHINSTANCE__@@QEAX@Z 0000000180007c04     MSVCRT:dll_dllmain.obj
 0002:00002c40       $unwind$?fin$0@?0??dllmain_crt_process_attach@@YAHQEAUHINSTANCE__@@QEAX@Z@4HA 0000000180007c40     MSVCRT:dll_dllmain.obj
 0002:00002c40       $unwind$?fin$0@?0??dllmain_crt_process_detach@@YAH_N@Z@4HA 0000000180007c40     MSVCRT:dll_dllmain.obj
 0002:00002c40       $unwind$?fin$1@?0??dllmain_crt_process_detach@@YAH_N@Z@4HA 0000000180007c40     MSVCRT:dll_dllmain.obj
 0002:00002c48       $unwind$?dllmain_crt_process_detach@@YAH_N@Z 0000000180007c48     MSVCRT:dll_dllmain.obj
 0002:00002c9c       $unwind$?dllmain_dispatch@@YAHQEAUHINSTANCE__@@KQEAX@Z 0000000180007c9c     MSVCRT:dll_dllmain.obj
 0002:00002cc4       $unwind$?filt$0@?0??dllmain_dispatch@@YAHQEAUHINSTANCE__@@KQEAX@Z@4HA 0000000180007cc4     MSVCRT:dll_dllmain.obj
 0002:00002ccc       $unwind$__scrt_is_nonwritable_in_current_image 0000000180007ccc     MSVCRT:utility.obj
 0002:00002cec       $unwind$__scrt_is_nonwritable_in_current_image$filt$0 0000000180007cec     MSVCRT:utility.obj
 0002:00002cf4       $unwind$__scrt_fastfail    0000000180007cf4     MSVCRT:utility_desktop.obj
 0002:00002d04       $unwind$__security_init_cookie 0000000180007d04     MSVCRT:gs_support.obj
 0002:00002d10       $unwind$__isa_available_init 0000000180007d10     MSVCRT:cpu_disp.obj
 0002:00002d20       $xdatasym                  0000000180007d20     MSVCRT:guard_dispatch.obj
 0002:00002d28       $xdatasym                  0000000180007d28     MSVCRT:guard_xfg_dispatch.obj
 0002:00002d30       .edata                     0000000180007d30     iterobjreachobj004.exp
 0002:00002d58       rgpv                       0000000180007d58     iterobjreachobj004.exp
 0002:00002d90       rgszName                   0000000180007d90     iterobjreachobj004.exp
 0002:00002dc8       rgwOrd                     0000000180007dc8     iterobjreachobj004.exp
 0002:00002de4       szName                     0000000180007de4     iterobjreachobj004.exp
 0002:00002dfb       $N00001                    0000000180007dfb     iterobjreachobj004.exp
 0002:00002e0a       $N00002                    0000000180007e0a     iterobjreachobj004.exp
 0002:00002e17       $N00003                    0000000180007e17     iterobjreachobj004.exp
 0002:00002e5c       $N00004                    0000000180007e5c     iterobjreachobj004.exp
 0002:00002e99       $N00005                    0000000180007e99     iterobjreachobj004.exp
 0002:00002ee1       $N00006                    0000000180007ee1     iterobjreachobj004.exp
 0002:00002f21       $N00007                    0000000180007f21     iterobjreachobj004.exp
 0002:00002f5e       $N00008                    0000000180007f5e     iterobjreachobj004.exp
 0002:00002f99       $N00009                    0000000180007f99     iterobjreachobj004.exp
 0002:00002fc7       $N00010                    0000000180007fc7     iterobjreachobj004.exp
 0002:00002ff8       $N00011                    0000000180007ff8     iterobjreachobj004.exp
 0002:00003027       $N00012                    0000000180008027     iterobjreachobj004.exp
 0002:00003056       $N00013                    0000000180008056     iterobjreachobj004.exp
 0002:0000308b       $N00014                    000000018000808b     iterobjreachobj004.exp
 0002:000034f2       .idata$6                   00000001800084f2     kernel32:KERNEL32.dll
 0002:00003556       .idata$6                   0000000180008556     vcruntime:VCRUNTIME140.dll
 0002:000036e8       .idata$6                   00000001800086e8     ucrt:api-ms-win-crt-heap-l1-1-0.dll
 0002:00003708       .idata$6                   0000000180008708     ucrt:api-ms-win-crt-runtime-l1-1-0.dll
 0002:0000372a       .idata$6                   000000018000872a     ucrt:api-ms-win-crt-convert-l1-1-0.dll
 0002:0000374c       .idata$6                   000000018000874c     ucrt:api-ms-win-crt-stdio-l1-1-0.dll
 0002:0000376c       .idata$6                   000000018000876c     ucrt:api-ms-win-crt-string-l1-1-0.dll
 0003:00000000       ?codeAttributeName@@3PEBDEB 0000000180009000     libiterobjreachobj004.obj
 0003:00000008       ?lineNumberAttributeName@@3PEBDEB 0000000180009008     libiterobjreachobj004.obj
 0003:00000010       ?localVarAttributeName@@3PEBDEB 0000000180009010     libiterobjreachobj004.obj
 0003:00000018       ?localVarTypeAttributeName@@3PEBDEB 0000000180009018     libiterobjreachobj004.obj
 0003:00000020       ?stackMapAttributeName@@3PEBDEB 0000000180009020     libiterobjreachobj004.obj
 0003:00000028       ?callBytes@@3PAEA          0000000180009028     libiterobjreachobj004.obj
 0003:0000002c       ?allocBytes@@3PAEA         000000018000902c     libiterobjreachobj004.obj
 0003:00000030       storage_data               0000000180009030     libiterobjreachobj004.obj
 0003:00000038       debugeeClassSignature      0000000180009038     libiterobjreachobj004.obj
 0003:00000040       objectFieldName            0000000180009040     libiterobjreachobj004.obj
 0003:0001aae4       redefineAttempted          0000000180023ae4     libiterobjreachobj004.obj
 0003:0001aae8       nsk_context                0000000180023ae8     libiterobjreachobj004.obj
 0003:0001aaf4       redefineSucceed            0000000180023af4     libiterobjreachobj004.obj
 0003:0001aaf8       agentFailed                0000000180023af8     libiterobjreachobj004.obj
 0003:0001aafc       currentAgentStatus         0000000180023afc     libiterobjreachobj004.obj
 0003:0001ab00       context                    0000000180023b00     libiterobjreachobj004.obj
 0003:0001abb8       agentThread                0000000180023bb8     libiterobjreachobj004.obj
 0003:0001abc0       agentThreadProc            0000000180023bc0     libiterobjreachobj004.obj
 0003:0001abc8       agentThreadArg             0000000180023bc8     libiterobjreachobj004.obj
 0003:0001abd0       agent_data                 0000000180023bd0     libiterobjreachobj004.obj
 0003:0001abe0       jvmti_env                  0000000180023be0     libiterobjreachobj004.obj
 0003:0001abe8       jvm                        0000000180023be8     libiterobjreachobj004.obj
 0003:0001abf0       jni_env                    0000000180023bf0     libiterobjreachobj004.obj
 0003:0001abf8       checkStatus_func           0000000180023bf8     libiterobjreachobj004.obj
 0003:0001ac00       ?codeAttributeIndex@@3GA   0000000180023c00     libiterobjreachobj004.obj
 0003:0001ac04       ?lineNumberAttributeIndex@@3GA 0000000180023c04     libiterobjreachobj004.obj
 0003:0001ac08       ?localVarAttributeIndex@@3GA 0000000180023c08     libiterobjreachobj004.obj
 0003:0001ac0c       ?localVarTypeAttributeIndex@@3GA 0000000180023c0c     libiterobjreachobj004.obj
 0003:0001ac10       ?stackMapAttributeIndex@@3GA 0000000180023c10     libiterobjreachobj004.obj
 0003:0001ac14       ?stackFrameOffset@@3GA     0000000180023c14     libiterobjreachobj004.obj
 0003:0001ac18       ?mode@@3HA                 0000000180023c18     libiterobjreachobj004.obj
 0003:0001ac1c       ?constantPoolSize@@3GA     0000000180023c1c     libiterobjreachobj004.obj
 0003:0001ac20       ?orig@@3PEBEEB             0000000180023c20     libiterobjreachobj004.obj
 0003:0001ac28       ?gen@@3PEAEEA              0000000180023c28     libiterobjreachobj004.obj
 0003:0001ac30       ?inputPos@@3PEAEEA         0000000180023c30     libiterobjreachobj004.obj
 0003:0001ac38       ?endPos@@3PEBEEB           0000000180023c38     libiterobjreachobj004.obj
 0003:0001ac40       ?genPos@@3PEAEEA           0000000180023c40     libiterobjreachobj004.obj
 0003:0001ac48       ?markPos@@3PEAEEA          0000000180023c48     libiterobjreachobj004.obj
 0003:0001ac50       ?constantPool@@3PEAPEADEA  0000000180023c50     libiterobjreachobj004.obj
 0003:0001ac58       ?constantPoolCount@@3GA    0000000180023c58     libiterobjreachobj004.obj
 0003:0001ac5c       ?zeroBytes@@3PAEA          0000000180023c5c     libiterobjreachobj004.obj
 0003:0001ac60       ?codeLength@@3IA           0000000180023c60     libiterobjreachobj004.obj
 0003:0001ac64       fakeUserData               0000000180023c64     libiterobjreachobj004.obj
 0003:0001ac68       ?map@@3PEAIEA              0000000180023c68     libiterobjreachobj004.obj
 0003:0001ac70       ?widening@@3PEACEA         0000000180023c70     libiterobjreachobj004.obj
 0003:0001ac78       timeout                    0000000180023c78     libiterobjreachobj004.obj
 0003:0001ac80       objCounter                 0000000180023c80     libiterobjreachobj004.obj
 0003:0001ac88       st_jvmti                   0000000180023c88     libiterobjreachobj004.obj
 0003:0001ac90       storage_ptr                0000000180023c90     libiterobjreachobj004.obj
 0003:0001aca0       GS_ExceptionRecord         0000000180023ca0     MSVCRT:gs_report.obj
 0003:0001ad40       GS_ContextRecord           0000000180023d40     MSVCRT:gs_report.obj
 0003:0001b210       ?g_tss_cv@@3U_RTL_CONDITION_VARIABLE@@A 0000000180024210     MSVCRT:thread_safe_statics.obj
 0003:0001b218       ?g_tss_event@@3PEAXEA      0000000180024218     MSVCRT:thread_safe_statics.obj
 0003:0001b220       ?g_tss_mutex@@3U_RTL_CRITICAL_SECTION@@A 0000000180024220     MSVCRT:thread_safe_statics.obj
 0003:0001b248       ?g_sleep_condition_variable_cs@@3P6AHPEAU_RTL_CONDITION_VARIABLE@@PEAU_RTL_CRITICAL_SECTION@@K@ZEA 0000000180024248     MSVCRT:thread_safe_statics.obj
 0003:0001b250       ?g_wake_all_condition_variable@@3P6AXPEAU_RTL_CONDITION_VARIABLE@@@ZEA 0000000180024250     MSVCRT:thread_safe_statics.obj
 0003:0001b25c       ?__proc_attached@@3HA      000000018002425c     MSVCRT:dll_dllmain.obj
 0003:0001b270       ?is_initialized_as_dll@@3_NA 0000000180024270     MSVCRT:utility.obj
 0003:0001b271       ?module_local_atexit_table_initialized@@3_NA 0000000180024271     MSVCRT:utility.obj
 0003:0001b278       ?module_local_atexit_table@@3U_onexit_table_t@@A 0000000180024278     MSVCRT:utility.obj
 0003:0001b290       ?module_local_at_quick_exit_table@@3U_onexit_table_t@@A 0000000180024290     MSVCRT:utility.obj
